:020000040800F2
:100000000028002021100008651000086510000875
:100010006510000865100008651000080000000069
:100020000000000000000000000000006510000853
:10003000651000080000000065100008FD0E0008B3
:1000400065100008651000086510000865100008BC
:1000500065100008651000086510000865100008AC
:10006000651000086510000865100008651000089C
:10007000651000086510000865100008651000088C
:10008000651000086510000865100008651000087C
:10009000651000086510000865100008651000086C
:1000A000651000086510000865100008651000085C
:1000B00065100008651000080000000065100008C9
:1000C0006510000800000000000000006510000836
:1000D0000000000065100008651000080000000026
:1000E0006510000865100008651000080000000099
:1000F0000000000000000000000000000000000000
:0C01000000000000000000005FF808F1A3
:10010C0080B483B000AF03463960FB7197F90730B8
:10011C00002B0BDA0D49FB7903F00F03043B3A6813
:10012C00D2B21201D2B20B441A7609E0084997F9FF
:10013C0007303A68D2B21201D2B20B4483F80023D2
:10014C0000BF0C37BD4680BC704700BF00ED00E01F
:10015C0000E100E080B582B000AF78607B68B3F15D
:10016C00807F01D3012311E00A4A7B6823F07F438F
:10017C00013B53600F214FF0FF30FFF7C1FF054BE0
:10018C0000229A60034B07221A6000231846083796
:10019C00BD4680BD10E000E080B500AF154A154BA0
:1001AC001B6843F0010313601249124B5A68124B3F
:1001BC0013404B600F4A0F4B1B6823F0847323F4DE
:1001CC00803313600B4A0B4B1B6823F480231360A2
:1001DC00084A084B5B6823F4FE035360054B4FF44D
:1001EC001F029A6000F078F8044B4FF000629A609E
:1001FC0000BF80BD001002400000FFF800ED00E0E1
:10020C0080B485B000AF0023FB600023BB600023EB
:10021C007B602C4B5B6803F00C03FB60FB68042BCE
:10022C0007D0082B09D0002B33D1274B274A1A6053
:10023C0033E0254B254A1A602FE0224B5B6803F410
:10024C007013BB601F4B5B6803F480337B60BB682F
:10025C009B0C0233BB607B68002B06D1BB681C4A2D
:10026C0002FB03F3184A136017E0164B5B6803F4A8
:10027C000033002B06D0BB68154A02FB03F3124A6D
:10028C0013600AE0BB68114A02FB03F30E4A1360C9
:10029C0003E00D4B0D4A1A6000BF0A4B5B6803F07C
:1002AC00F0031B090B4AD35CDBB2FB60064B1A68EC
:1002BC00FB6822FA03F3044A136000BF1437BD46EF
:1002CC0080BC7047001002400000002000127A0031
:1002DC0000093D000400002080B500AF00F002F8DA
:1002EC0000BF80BD80B483B000AF00237B600023CF
:1002FC003B603A4A394B1B6843F480331360374BED
:10030C001B6803F400333B607B6801337B603B6804
:10031C00002B03D17B68B3F5A06FF0D12F4B1B687A
:10032C0003F40033002B02D001233B6001E00023D7
:10033C003B603B68012B4BD1294A294B1B6843F08E
:10034C0010031360264A264B1B6823F0030313602B
:10035C00234A234B1B6843F0020313601F4A1F4BB5
:10036C005B6853601D4A1D4B5B6853601B4A1B4BFB
:10037C005B6843F480635360184A184B5B6823F442
:10038C007C135360154A154B5B6843F4E8135360B8
:10039C00124A124B1B6843F08073136000BF0F4B63
:1003AC001B6803F00073002BF9D00C4A0B4B5B68F5
:1003BC0023F003035360094A084B5B6843F00203C4
:1003CC00536000BF054B5B6803F00C03082BF9D19D
:1003DC0000BF0C37BD4680BC704700BF0010024008
:1003EC000020024080B489B000AF786039600023EF
:1003FC00FB6100233B610023BB610023FB600023F6
:10040C007B610023BB603B68DB7803F00F03FB616F
:10041C003B68DB7803F01003002B05D03B689B781E
:10042C001A46FB691343FB613B681B88DBB2002B4C
:10043C0044D07B681B687B610023BB6138E00122E0
:10044C00BB6902FA03F3FB603B681B881A46FB6826
:10045C0013403B613A69FB689A4226D1BB699B0009
:10046C00FB600F22FB6802FA03F3BB60BB68DB4343
:10047C007A6913407B61FA69FB6802FA03F37A69C3
:10048C0013437B613B68DB78282B05D10122BB69C8
:10049C009A407B685A6108E03B68DB78482B04D1B2
:1004AC000122BB699A407B681A61BB690133BB614D
:1004BC00BB69072BC3D97B687A691A603B681B88B8
:1004CC00FF2B46D97B685B687B610023BB613AE0FC
:1004DC00BB690833012202FA03F3FB603B681B88FB
:1004EC001A46FB6813403B613A69FB689A4227D174
:1004FC00BB699B00FB600F22FB6802FA03F3BB6035
:10050C00BB68DB437A6913407B61FA69FB6802FACA
:10051C0003F37A6913437B613B68DB78282B05D1A5
:10052C00BB69083301229A407B685A613B68DB78CF
:10053C00482B05D1BB69083301229A407B681A61AC
:10054C00BB690133BB61BB69072BC1D97B687A6975
:10055C005A6000BF2437BD4680BC704780B483B05E
:10056C0000AF78600B467B807A887B681A6100BF8D
:10057C000C37BD4680BC704780B483B000AF786048
:10058C000B467B807A887B685A6100BF0C37BD466E
:10059C0080BC704780B483B000AF78600B46FB70B2
:1005AC00FB78002B06D00949084B9A697B681343EA
:1005BC008B6106E00549054B9A697B68DB43134068
:1005CC008B6100BF0C37BD4680BC704700100240E9
:1005DC0080B485B000AF78600B467B800023FB7342
:1005EC007B681B899AB27B8813409BB2002B02D08C
:1005FC000123FB7301E00023FB73FB7B18461437CC
:10060C00BD4680BC704700BF80B483B000AF78603B
:10061C000B467B807B687A889A8100BF0C37BD467D
:10062C0080BC704780B483B000AF78607B689B89D6
:10063C009BB218460C37BD4680BC704780B485B061
:10064C0000AF786039600023FB817B681B88FB81DD
:10065C00FB8903F44153FB813B681A883B685B8838
:10066C0013439AB23B689B8813439AB23B68DB886E
:10067C0013439AB23B681B8913439AB23B685B895C
:10068C0013439AB23B689B8913439AB23B68DB894C
:10069C0013439AB2FB891343FB817B68FA891A8056
:1006AC007B689B8B9BB223F400639AB27B689A8322
:1006BC003B681A8A7B681A8200BF1437BD4680BC1F
:1006CC00704700BF80B483B000AF78600B46FB70FE
:1006DC00FB78002B08D07B681B889BB243F040034F
:1006EC009AB27B681A8007E07B681B889BB223F068
:1006FC0040039AB27B681A8000BF0C37BD4680BCA1
:10070C00704700BF80B483B000AF78600B46FB70BD
:10071C00FB78002B06D07B689B6843F001027B685A
:10072C009A6005E07B689B6823F001027B689A6005
:10073C0000BF0C37BD4680BC704700BF80B483B08F
:10074C0000AF78607B689B6843F008027B689A6016
:10075C0000BF0C37BD4680BC704700BF80B485B06D
:10076C0000AF78600023FB737B689B6803F0080381
:10077C00002B02D00123FB7301E00023FB73FB7BF6
:10078C0018461437BD4680BC704700BF80B483B098
:10079C0000AF78607B689B6843F004027B689A60CA
:1007AC0000BF0C37BD4680BC704700BF80B485B01D
:1007BC0000AF78600023FB737B689B6803F0040335
:1007CC00002B02D00123FB7301E00023FB73FB7BA6
:1007DC0018461437BD4680BC704700BF80B483B048
:1007EC0000AF78600B46FB70FB78002B06D07B6863
:1007FC009B6843F4A0027B689A6005E07B689B6869
:10080C0023F4A0027B689A6000BF0C37BD4680BC05
:10081C00704700BF80B485B000AF786039600023AA
:10082C00FB600023FB727B685B68FB60FB6803F476
:10083C004153FB603B681A683B681B791B021343EE
:10084C00FA681343FB607B68FA685A607B689B68A4
:10085C00FB60FA68164B1340FB603B68DA683B6838
:10086C009B681A433B685B795B001343FA6813433C
:10087C00FB607B68FA689A607B68DB6AFB60FB68EC
:10088C0023F47003FB603B681B7C013BDAB2FB7A00
:10089C001343FB72FB7A1B05FA681343FB607B68FE
:1008AC00FA68DA6200BF1437BD4680BC704700BFDF
:1008BC00FDF7F1FF80B483B000AF78607B68DB6C30
:1008CC009BB218460C37BD4680BC704780B582B0D1
:1008DC0000AF0346FB7100BF02210E48FFF778FE04
:1008EC000346002BF8D0FB799BB219460948FFF759
:1008FC008BFE00BF01210748FFF76AFE0346002B61
:10090C00F8D00448FFF78EFE0346DBB218460837D2
:10091C00BD4680BD0030014080B586B000AF0121DE
:10092C000420FFF737FE01214FF48050FFF732FE11
:10093C00E023BB820323BB751823FB7507F114035B
:10094C0019461748FFF74EFD1023BB821023FB7589
:10095C0007F1140319461248FFF744FD00233B80AE
:10096C004FF482737B800023BB800223FB80012326
:10097C003B814FF400737B810023BB810023FB81FF
:10098C0007233B823B4619460648FFF757FE0121D9
:10099C000448FFF797FE00BF1837BD4680BD00BF67
:1009AC00000801400030014080B500AF102118480C
:1009BC00FFF7E2FD95220021002000F02BF801202A
:1009CC0000F05EF80346002B01D0FF231DE0102140
:1009DC000F48FFF7C3FDFF20FFF778FF10210C48ED
:1009EC00FFF7CAFDFF220021012000F013F80020C0
:1009FC0000F046F80346002BE9D110210448FFF71C
:100A0C00ADFDFF20FFF762FF0023184680BD00BF3D
:100A1C000008014080B586B000AF03463960FB7119
:100A2C001346BB7100237B61FB7943F04003DBB2BF
:100A3C003B733B681B0EDBB27B733B681B0CDBB25E
:100A4C00BB733B681B0ADBB2FB733B68DBB23B74CA
:100A5C00BB797B7400237B610AE007F10C027B6994
:100A6C0013441B781846FFF731FF7B6901337B6118
:100A7C007B69052BF1D900BF1837BD4680BD00BF7F
:100A8C0080B584B000AF0346FB7140F6FF73FB608A
:100A9C0002E0FB68013BFB6000F012F803461A46CB
:100AAC00FB79934202D0FB68002BF2D1FB68002B40
:100ABC0001D1FF2300E0002318461037BD4680BD4E
:100ACC0080B582B000AF0023FB7100BF02210E483D
:100ADC00FFF77EFD0346002BF8D0FF210A48FFF7F5
:100AEC0093FD00BF01210848FFF772FD0346002B60
:100AFC00F8D00548FFF796FD0346FB71FB791846C5
:100B0C000837BD4680BD00BF0030014080B582B0C3
:100B1C0000AF00237B601EE0FFF7D2FF0346FB70A3
:100B2C00FB7803F01F03FB70FB780B2B06D00D2B0F
:100B3C0006D0052B06D10523BB7006E00B2316E06F
:100B4C000D2314E0FF23BB7000BFBB78052B06D030
:100B5C007B6801337B607B68402BDDD900E000BFF4
:100B6C0000BFFFF7ADFF0346002BFAD0FB78184609
:100B7C000837BD4680BD00BF80B582B000AF0023F2
:100B8C007B60FFF7C9FE10210A48FFF7E7FC002342
:100B9C007B6005E0FF20FFF799FE7B6801337B60EB
:100BAC007B68092BF6D9FFF7FFFE0346184608377A
:100BBC00BD4680BD0008014080B500AF094B1B88C5
:100BCC00002B01D100230AE0FFF7D6FF03469AB2AF
:100BDC00044B1A80034B1B88002BF5D101231846BC
:100BEC0080BD00BF1800002080B500AF00BFFFF72C
:100BFC00E3FF0346002BFAD100BF80BD80B586B061
:100C0C0000AFF860B9601346FB8000237B61FF23C3
:100C1C00FB7410211E48FFF7AFFCFF22B9681820A7
:100C2C00FFF7F8FE0020FFF72BFF0346002B22D125
:100C3C00FF20FFF74BFEFE20FFF748FE00237B61F1
:100C4C000AE0FB681B781846FFF740FEFB6801338F
:100C5C00FB607B6901337B61FA887B699A42F0D82F
:100C6C00FFF72EFFFFF72CFFFFF750FF0346052B76
:100C7C0001D10023FB7410210548FFF76FFCFF2006
:100C8C00FFF724FEFB7C18461837BD4680BD00BF1D
:100C9C000008014080B584B000AF78603B4B1A78F7
:100CAC003B4B1A70394B00221A700023FB60FF2358
:100CBC00FB7210213748FFF75FFCFF227968182080
:100CCC00FFF7A8FE0020FFF7DBFE0346002B4ED1FA
:100CDC00FF20FFF7FBFDFE20FFF7F8FD2C4B1B78E8
:100CEC00012B1AD10023FB6014E02B4AFB6832F86D
:100CFC001330DBB21846FFF7E9FD274AFB6832F8E0
:100D0C0013301B0A9BB2DBB21846FFF7DFFDFB6802
:100D1C000133FB60FB68FF2BE7D91D4B1B78022BC3
:100D2C001AD10023FB6014E01C4AFB6832F8133024
:100D3C00DBB21846FFF7CAFD184AFB6832F81330CD
:100D4C001B0A9BB2DBB21846FFF7C0FDFB680133F0
:100D5C00FB60FB68FF2BE7D9FFF7B2FEFFF7B0FE95
:100D6C00FFF7D4FE0346052B01D10023FB721021A3
:100D7C000848FFF7F3FBFF20FFF7A8FD044B002208
:100D8C001A70FB7A18461037BD4680BD300600201D
:100D9C001B0000200008014030020020300400201D
:100DAC0080B586B000AF01214FF40070FFF7F2FB65
:100DBC0001233B800023FB700223BB703B4619468A
:100DCC001A48FFF70FFB00237B6001233B720123C2
:100DDC007B724FF46023FB6000233B6100233B7567
:100DEC003B1D19461248FFF715FD01211048FFF76E
:100DFC0089FC0F48FFF7A2FC00BF0D48FFF7AEFCC3
:100E0C000346002BF9D10A48FFF7C0FC00BF084885
:100E1C00FFF7CCFC0346002BF9D101210448FFF766
:100E2C00DDFC00BF1837BD4680BD00BF0008014087
:100E3C000024014080B500AF4FF400720021094836
:100E4C0000F084F923220849064800F007F9002035
:100E5C00FFF720FF03469AB2044B1A800123184671
:100E6C0080BD00BF300200204C120008180000208A
:100E7C0080B500AFFFF780FE03461A46154B1A608B
:100E8C00FFF7B2FE144B00221A80144B4FF4007281
:100E9C001A60FFF7B5F9124B1B68124AA2FB032329
:100EAC001B0B1846FFF756F9FFF77AFF0E4B1B7812
:100EBC00002BFBD00D4B01221A70084B1B681846F7
:100ECC00FFF7E8FE054B1B6803F50073034A13603C
:100EDC00ECE700BF140000202602002028020020AE
:100EEC00000000205917B7D1300600203206002030
:100EFC0080B500AF3948FFF7DDFC03461A46384B86
:100F0C001A80384B1B78012B30D1374B1B78012BB7
:100F1C002CD0364B1B781A46354B1988354B23F899
:100F2C001210324B1B780133DAB2304B1A702F4B44
:100F3C001B781A462A4B1B8899B22E4B23F8121099
:100F4C002A4B1B780133DAB2284B1A70284B1B88BA
:100F5C0001339AB2264B1A80244B1B78002B05D1F7
:100F6C00204B02221A70244B01221A701D4B1B7845
:100F7C00022B30D11C4B1B78022B2CD01B4B1B781B
:100F8C001A461B4B19881D4B23F81210174B1B7854
:100F9C000133DAB2154B1A70144B1B781A46104BEE
:100FAC001B8899B2154B23F81210104B1B78013388
:100FBC00DAB20E4B1A700E4B1B8801339AB20C4BE3
:100FCC001A800A4B1B78002B05D1064B01221A7094
:100FDC00094B02221A7000BF80BD00BF00240140E3
:100FEC002C0200201A0000201B00002031060020DB
:100FFC00340600203002002030060020300400208F
:10100C0070120008000000201C0000201C000020B2
:10101C0038060020002103E00A4B5B584350043192
:10102C0009480A4B42189A42F6D3094A02E00023B7
:10103C0042F8043B074B9A42F9D3FFF7ADF8FFF7A0
:10104C0017FF704770120008000000201C000020E1
:10105C001C00002038060020FEE700000F0052E3C1
:10106C00F0402DE92900009A003081E1030013E3E0
:10107C003100001A02E0A0E110C080E2103081E2E1
:10108C00107013E50C6013E5085013E5044013E5EC
:10109C0010E04EE20F005EE310700CE50C600CE506
:1010AC0008500CE504400CE5103083E210C08CE2D3
:1010BC00F2FFFF8A103042E20F30C3E30F6002E20E
:1010CC00103083E2030056E3031081E0033080E02C
:1010DC001B00009A0140A0E106C0A0E104E043E23D
:1010EC0004C04CE2045094E403005CE30450AEE50D
:1010FC00FAFFFF8A04C046E203C0CCE304C08CE2D2
:10110C000C3083E00C1081E0032002E2000000EAC6
:10111C000030A0E1000052E30500000A013043E278
:10112C00022081E001C0D1E4020051E101C0E3E5FD
:10113C00FBFFFF1AF040BDE81EFF2FE10030A0E1DD
:10114C00F5FFFFEA0620A0E1F1FFFFEA030010E340
:10115C0010402DE93700000A000052E3012042E262
:10116C003200000AFFC001E20030A0E1020000EAF8
:10117C00000052E3012042E22C00000A01C0C3E44B
:10118C00030013E3F9FFFF1A030052E32000009A57
:10119C00FFE001E20EE48EE10F0052E30EE88EE177
:1011AC001000009A0240A0E110C083E2104044E21B
:1011BC000F0054E310E00CE50CE00CE508E00CE546
:1011CC0004E00CE510C08CE2F7FFFF8A10C042E28D
:1011DC000FC0CCE30F2002E210C08CE2030052E3FC
:1011EC000C3083E00A00009A0340A0E102C0A0E1A9
:1011FC0004C04CE203005CE304E084E4FBFFFF8AE0
:10120C0004C042E203C0CCE304C08CE20C3083E0A7
:10121C00032002E2000052E3FF10011202208310AF
:10122C000200000A0110C3E4020053E1FCFFFF1AA4
:10123C001040BDE81EFF2FE10030A0E1D1FFFFEA16
:10124C0000766F6C746C6F6767657200010100004B
:10125C00566F6C746C6F676765723030303000306D
:04126C00003000004E
:1012700000A24A0400000000000000000102030474
:0C128000060708090A000000FFFF010239
:0400000508001021BE
:00000001FF
